:020000040800F2
:1000000000060020A1020008E90F0008ED0F00081B
:1000100045100008ED0F000819100008A3020008A1
:10002000A3020008A3020008A3020008592900083F
:10003000A3020008A3020008A3020008A30200080C
:10004000A3020008A3020008A3020008A3020008FC
:10005000A3020008A3020008D93D0008053E0008DD
:10006000313E00085D3E0008893E0008A3020008FA
:10007000A3020008A3020008A3020008A3020008CC
:10008000A3020008A3020008A3020008A3020008BC
:10009000A3020008A3020008A3020008B53E00085E
:1000A000A3020008A3020008A3020008A30200089C
:1000B000A3020008A3020008A3020008A30200088C
:1000C000A3020008A3020008A3020008A30200087C
:1000D000A3020008A3020008A3020008A30200086C
:1000E000193F0008A3020008A3020008A3020008A9
:1000F000A3020008A3020008A3020008A30200084C
:10010000A3020008A3020008A13F0008A302000800
:10011000A3020008A3020008A3020008A30200082B
:10012000A3020008A3020008A3020008A30200081B
:10013000A3020008A3020008A3020008A30200080B
:10014000A3020008A3020008A3020008A3020008FB
:10015000A3020008A3020008A3020008A3020008EB
:10016000A3020008A3020008A3020008A3020008DB
:10017000A3020008F9340008A3020008A302000843
:10018000A3020008A30200088D3F0008A302000894
:10019000A3020008A3020008A3020008A3020008AB
:1001A000A3020008A3020008A3020008A30200089B
:1001B000A3020008A3020008A3020008A30200088B
:1001C000A3020008A3020008A3020008A30200087B
:1001D000A3020008E5340008A3020008A3020008F7
:1001E000A3020008A3020008A3020008A30200085B
:1001F000A3020008A3020008A3020008A30200084B
:10020000A3020008A3020008A3020008A30200083A
:10021000A3020008A3020008A3020008A30200082A
:10022000A3020008A3020008A3020008A30200081A
:10023000A3020008A3020008A3020008A30200080A
:10024000A3020008A3020008A3020008A3020008FA
:10025000A3020008A3020008A3020008A3020008EA
:10026000A3020008A3020008A3020008A3020008DA
:10027000A3020008A3020008A3020008A3020008CA
:10028000A3020008A3020008A3020008A3020008BA
:10029000A3020008A3020008A3020008A3020008AA
:1002A00002E000F000F8FEE772B6394880F30888F3
:1002B000384880F3098838484EF60851CEF20001DC
:1002C000086040F20000CCF200004EF63471CEF22D
:1002D00000010860BFF34F8FBFF36F8F40F2000043
:1002E000C0F2F0004EF68851CEF200010860BFF374
:1002F0004F8FBFF36F8F4FF00000E1EE100A4EF604
:100300003C71CEF200010860062080F31488BFF330
:100310006F8F02F085FB03F039FB4FF055301F491A
:100320001B4A91423CBF41F8040BFAE71C49194AA9
:1003300091423CBF41F8040BFAE71A491A4A1B4B99
:100340009A423EBF51F8040B42F8040BF8E7002034
:100350001749184A91423CBF41F8040BFAE702F0F2
:10036000A3FB03F093FB144C144DAC4203DA54F896
:10037000041B8847F9E700F041F8114C114DAC42DD
:1003800003DA54F8041B8847F9E702F08BBB00003E
:1003900000060020002200200000000800000020CD
:1003A00000060020A843000800220020442200206C
:1003B00048220020F0460020A0020008A002000809
:1003C000A0020008A00200082DE9F04F2DED108AD0
:1003D000C1F80CD0D0F80CD0BDEC108ABDE8F08F7D
:1003E000002383F311882846A047002001F0B0FEC7
:1003F000FEE701F031FE00DFFEE7000038B51F4CDC
:100400000523002523700423A57063701E23E57067
:1004100025716571A571E57125726572A372E5722A
:1004200000F0E2FC20B10E2325726572A372E57222
:1004300002F054FA044602F089FA0546D0B9104B8E
:100440009C4219D001339C4241F2883412BF0546C8
:1004500000240125002002F04BFA0DB100F05AF8FB
:1004600000F068FD00F008FC204600F013F900F0F1
:1004700051F8F9E70024EDE70446EBE748220020B5
:10048000010007B008B500F0C3FBA0F120035842FB
:10049000584108BD054B07B51B88022101A8ADF8DE
:1004A000043000F0D3FB03B05DF804FB5C400008AF
:1004B00010B5202383F311881248C3680BB101F0F3
:1004C000E3FE0023104A4FF47A710E4801F08AFED1
:1004D000002383F311880D4C236813B12368013B7B
:1004E0002360636813B16368013B6360084B1B784A
:1004F00033B9636823B9022000F08CFC32236360B7
:1005000010BD00BF54220020B10400087023002059
:1005100068220020554B56492DE9F04153F8042F2D
:10052000013201D1BDE8F0818B42F7D1514C524BE1
:1005300022689A4240F29880504B9B6803F1006316
:1005400003F500339A4280F08F80002000F0B0FB6A
:1005500002204B4B187000F053FC4A4BD3F8E820B4
:100560000022C3F8E820D3F81011C3F81021D3F803
:100570001011D3F8EC10C3F8EC20D3F81411C3F821
:100580001421D3F81411D3F8F010C3F8F020D3F8E5
:100590001811C3F81821D3F81811D3F8801041F0BE
:1005A0000061C3F88010D3F8801021F00061C3F817
:1005B0008010D3F88010D3F8801041F00071C3F898
:1005C0008010D3F8801021F00071C3F88010D3F8A8
:1005D000803072B62C4B2D490B601D682468BFF328
:1005E0004F8FBFF36F8F2A4BC3F88420BFF34F8F19
:1005F0005A6922F480325A61BFF34F8FD3F88020BA
:1006000043F6E07EC2F3C906C2F34E32B707520189
:1006100002EA0E0838463146013948EA000C00F17A
:100620004040B1F1FF3FC3F874C2F5D1203A12F156
:10063000200FEDD1BFF34F8FBFF36F8FBFF34F8FFD
:10064000BFF36F8F5A6922F400325A610022C3F857
:100650005022BFF34F8FBFF36F8F202383F3118896
:10066000AD4685F308882047BDE8F081FCFF01080E
:100670001C00020804000208FFFF010848220020B5
:1006800068220020004402580000020808ED00E043
:1006900000ED00E02DE9F04F99B0B34C2022FF218E
:1006A000019010A8A66800F0E7FBB04AA3461378B3
:1006B000A3B90121AE481170C360202383F31188D0
:1006C000C3680BB101F0E0FD0023AA4A4FF47A7130
:1006D000A74801F087FD002383F31188019B13B124
:1006E000A54B019A1A600023A44AA349019F994689
:1006F0001C461D46984613704B600292012000F084
:100700007FFB002F00F012829B4B1B68002B40F0F8
:100710000D8219B0BDE8F08F0220FFF7B3FE00286C
:1007200040F0FB81019BB9F1000F08BF1F46944BBD
:100730001B8802210BA8ADF82C3000F087FADDE70A
:100740004FF47A7000F064FA031E0393EADB022090
:10075000FFF798FE82460028E4D0039B581E042829
:1007600000F2DD81DFE800F0030E1114170018A875
:100770000523042140F8343D00F068FA54464FF058
:10078000000856E004217848F6E704217D48F3E7A5
:1007900004217D48F0E71C242046043400F08AFA46
:1007A00004210B900BA800F051FA2C2CF4D1E5E7B2
:1007B000002DB7D0002CB5D00220FFF763FE054610
:1007C000002800F0AF8101206C4C00F071FA4FF06E
:1007D00000090220207000F013FB5FFA89FA5046EE
:1007E00000F076FA074658B1504609F1010900F0C9
:1007F0007FFA0028F1D12C46A9460027634B97E7E2
:1008000001233E460220237000F0F0FADBF80830A6
:100810009E4206D2304600F04DFA0130EBD104364C
:10082000F4E70026029BA9462C461E703746524B21
:100830005E6000F075FB15B1002C18BF0027FFF7B4
:1008400029FE5BE7002D3FF46DAF002C3FF46AAF4B
:100850000220029B187000F0D3FA322000F0D8F981
:10086000B0F1000AC0F25E811AF0030540F05A812F
:1008700006EB0A03DBF80820934200F25381BAF535
:10088000807F00F24F8155450DDA4FF47A7000F009
:10089000BFF90490049B002BC0F24481049B3C4AA6
:1008A000AB540135EFE7C820FFF7ECFD0546002803
:1008B00000F038811F2E11D8C6F1200410AB26F0AD
:1008C000030033495445184428BF5446224600F0DB
:1008D000ABFA2246FF212E4800F0CEFA4FEAAA0AD0
:1008E0002B4930465FFA8AF200F0CEFA044600281F
:1008F00000F01A8106EB8A0605469AE70220FFF708
:10090000C1FD00283FF40EAF00F00CFA00283FF4C0
:1009100009AF4FF0000A5346DBF8082092451CD27D
:10092000BAF11F0F12D8109A01320FD02AF0030229
:1009300018A90A4452F8202C0B92184604220BA93D
:100940000AF1040A00F092FB0346E5E750460393E0
:1009500000F0B0F9039B0B90EFE718A8042140F8D2
:100960004C3D00F073F964E7482200206C2300201E
:1009700054220020B10400087023002068220020C7
:100980005E4000084C2200205022002060400008F9
:100990006C22002018A80023642140F8343D00F0A8
:1009A0004BF900287FF4BEAE0220FFF76BFD002854
:1009B0003FF4B8AE0B9800F0ADF918AB43F8480D12
:1009C00004211846CDE718A80023642140F8343DDF
:1009D00000F032F900287FF4A5AE0220FFF752FDA7
:1009E00000283FF49FAE0B9800F096F918AB43F83F
:1009F000440DE5E70220FFF745FD00283FF492AEE5
:100A000000F0A0F918AB43F8400DD9E70220FFF73A
:100A100039FD00283FF486AE0BA9142000F098F9A8
:100A2000824618A8042140F83CAD00F00FF9514669
:100A30000BA896E7322000F0EBF8B0F1000AFFF6C1
:100A400071AE1AF0030F7FF46DAE0AEB0803DBF80A
:100A5000082093423FF666AE0220FFF713FD002800
:100A60003FF460AE2AF0030AC244D0453FF4E1AE41
:100A7000404608F1040800F01DF904210A900AA874
:100A800000F0E4F8F1E74FF47A70FFF7FBFC002880
:100A90003FF448AE00F046F900283FF4AFAE109B9B
:100AA00001330CD0082210A9002000F0EDF9002835
:100AB0003FF4A4AE2022FF2110A800F0DDF9FFF7DB
:100AC000E9FC374801F04AFB23E6002D3FF42AAE4B
:100AD000002C3FF427AE18A80023642140F8343DD1
:100AE00000F0AAF8824600287FF41CAE0220FFF72F
:100AF000C9FC00283FF416AE0390FFF7CBFC41F28F
:100B00008830574601F02AFB0B9800F04DFA00F0B0
:100B100007FA039B1C461D46F0E5054689E64FF0A3
:100B20000008FFE52546FDE52C4667E6002000F0BD
:100B30006FF80490049B002BFFF6E3AD012000F05A
:100B400055F9049B213B122B3FF6D8AD01A252F878
:100B500023F000BF1907000841070008B10700088B
:100B6000FD060008FD060008FD060008450800080F
:100B7000350A0008FD08000895090008C7090008A3
:100B8000F5090008FD0600080D0A0008FD0600082A
:100B9000870A000833080008FD060008CB0A000891
:100BA000A08601002DE9F84F4FF47A7507460E46EE
:100BB00000245543DFF85080DFF8509098F900305A
:100BC0005FFA84FA5A1C01D0A34210D159F82400CC
:100BD000324639460368D3F820B02B46D8478642C0
:100BE00005D1084B012083F800A0BDE8F88F01343F
:100BF000022CE3D14FF4FA7001F0B0FA0020BDE806
:100C0000F88F00BFBC2300200022002064400008B1
:100C100007B5002202AB012103F8012D0246184658
:100C2000FFF7C0FF20B19DF8070003B05DF804FB9B
:100C30004FF0FF30F9E700000A46042108B5FFF73E
:100C4000B1FF80F00100C0B2404208BD074B30B494
:100C50001A78074B53F822400A460146236820467B
:100C6000DD69044BAC4630BC604700BFBC230020AC
:100C700064400008A0860100F8B50A4C00250A4E21
:100C800001F012FD094F208030682388834207D984
:100C900001F006FD336805440133BD423360F3D9EA
:100CA000F8BD00BFBE23002078230020FFFF010015
:100CB00001F0C8BD00F1006000F500300068704729
:100CC00000F10060920000F5003001F049BD000025
:100CD000054B1A68054B1B889B1A834202D91044A6
:100CE00001F0DEBC0020704778230020BE230020E6
:100CF00038B5074D04462868204401F0D7FC28B9D0
:100D000028682044BDE8384001F0E2BC38BD00BF8F
:100D10007823002000207047014BC058704700BF67
:100D200000E8F11F064991F8243033B1002308226E
:100D3000086A81F82430FFF7C3BF0120704700BF65
:100D40007C230020014B1868704700BF0010005C36
:100D5000234BF0B5234C1B682788C3F30B0665684B
:100D60001B0C94F90820BE4228D0A789BE4206D1A8
:100D700001220C2505FB0244656894F9082041F224
:100D80000104A3421CD041F20304A3421AD042F250
:100D90000104A34218D042F20304A34208BF562222
:100DA000441E013D0B460C44A34217D215F9016FB6
:100DB000581C5EB1034600F8016CF5E70022D8E745
:100DC0005A22EDE75922EBE75822E9E72C25844225
:100DD0001D7001D9981C5A70401AF0BD1846FBE7E7
:100DE0000010005C0422002000207047022803D17C
:100DF0004FF00062014B9A61704700BF0004025837
:100E0000022803D14FF40062014B9A61704700BF82
:100E100000040258022804D1024A536983F4006393
:100E20005361704700040258002310B5934203D069
:100E3000CC5CC4540133F9E710BD000030B5441E4A
:100E400014F9010F0B4658B193F900500131854256
:100E500006D11AB993F90020801A30BD013AEFE7A4
:100E6000002AF7D1104630BD02460346981A13F9FE
:100E7000011B0029FAD1704702440346934202D075
:100E800003F8011BFAE770472DE9F047234C0546AC
:100E90008846174694F8243083BB2E46DFF87C90B2
:100EA000C7B394F824302BB92022FF21484626628C
:100EB000FFF7E2FF94F824004146C0F1080504EB77
:100EC0008000BD4228BF3D465FFA85FAAD00A7EB22
:100ED0000A072A462E44FFF7A7FF94F82430A844B7
:100EE000FFB29A445FFA8AFABAF1080F84F824A094
:100EF000D6D1FFF717FF0028D2D108E0266A06EB0B
:100F00008306B042CAD0FFF70DFF0028C5D10020EC
:100F1000BDE8F0870120BDE8F08700BF7C230020FA
:100F2000024B1A78024B1A70704700BFBC23002096
:100F30000022002038B5164C164D204600F00CFC5F
:100F40002946204600F034FC2D681348D5F890203F
:100F5000D2F8043843F00203C2F8043801F0FEF876
:100F60000E49284600F036FDD5F890200C48D2F8FE
:100F700004380C49A04223F00203C2F804384FF4AD
:100F8000E1330B6003D0BDE8384000F043BB38BD0F
:100F9000682A00206C41000840420F00944100087C
:100FA00040240020A423002038B50B4B05461A78B6
:100FB0000A4B53F822400A4B9C420CD0094B0021AB
:100FC00018221846FFF758FF056001462046BDE885
:100FD000384000F01FBB38BDBC230020644000082F
:100FE000682A0020A4230020FEE7000000B59BB083
:100FF000EFF3098168226846FFF716FFEFF30583D8
:10100000044B9A6BDA6A9A6A9A6A9A6A9A6A9A6A34
:101010009B6AFEE700ED00E000B59BB0EFF30981AD
:1010200068226846FFF700FFEFF30583044B9A6BD5
:101030009A6A9A6A9A6A9A6A9A6A9B6AFEE700BFF3
:1010400000ED00E000B59BB0EFF30981682268462F
:10105000FFF7EAFEEFF30583034B5A6B9A6A9A6A2D
:101060009A6A9A6A9B6AFEE700ED00E030B50A448E
:10107000074D91420BD011F8013B09245840013C27
:10108000F7D040F300032B4083EA5000F7E730BD70
:101090002083B8ED002304491A465A50C818083373
:1010A0004260802BF9D17047C0230020026843685A
:1010B0001143016003B1184770470000024A1368EA
:1010C00043F0C003136070470078004013B50E4C26
:1010D000204600F093FA04F11400009400234FF42A
:1010E00000720A4900F054F90094094B4FF4007261
:1010F000084904F1380000F0CDF9074BE365074BD0
:10110000236602B010BD00BF40240020AC240020A4
:10111000BD100008AC2600200078004000E1F50575
:10112000254B002908BF1946037C012B30B511D18E
:10113000224B98420ED1224BD3F8E82042F0804255
:10114000C3F8E820D3F8102142F08042C3F8102100
:10115000D3F810310A68036EC46D03EB5203816645
:10116000B3FBF2F34A68150442BF23F0070503F00E
:10117000070343EA4503E3608B6843F04003636081
:10118000CB68510543F00103A36042F4967343F02A
:10119000010323604FF0FF33236205D512F01022C4
:1011A00005D0B2F1805F04D080F8643030BD7F2379
:1011B000FAE73F23F8E700BF8840000840240020FA
:1011C000004402582DE9F047C66D05463768F469BA
:1011D000200734621AD014F0080F0CBF00218021C0
:1011E000E20748BF41F02001A3074FF0200348BFAA
:1011F00041F04001600748BF41F4807183F31188DA
:10120000281DFFF753FF002383F31188E2050AD559
:10121000202383F311884FF40071281DFFF746FF48
:10122000002383F311884FF020094FF0000A14F0D7
:10123000200831D13B0616D54FF0200905F1380AB8
:10124000200610D589F31188504600F057F9002880
:101250002FDA0821281DFFF729FF27F080033360CC
:10126000002383F3118879060DD562060BD5202360
:1012700083F31188EA6C2B6D9A4201D12B6CEBB988
:10128000002383F31188E30620D5AA6E1369EBB11E
:101290005069BDE8F047184789F31188736A2846FA
:1012A00095F86410194000F0C3F98AF31188F469C5
:1012B000BDE7B06288F31188F469C1E727F0400701
:1012C0001021281DFFF7F2FE3760D9E7BDE8F0874F
:1012D000F8B51546826804460B46AA4200D28568D6
:1012E000A1692669761AB54207D218462A46FFF741
:1012F0009BFDA3692B44A3610DE011D9AF1B3246BE
:101300001846FFF791FD3A46E1683044FFF78CFD3F
:10131000E2683A44A261A36828465B1BA360F8BD5B
:1013200018462A46FFF780FDE368E4E783689342A6
:101330002DE9F04104460F46154600D285686069E4
:101340002669361AB54207D22A463946FFF76CFDA0
:1013500063692B4463610EE013D9A5EB060832469E
:101360003946FFF761FD4246B919E068FFF75CFDB9
:10137000E26842446261A36828465B1BA360BDE843
:10138000F0812A463946FFF74FFDE368E2E70000A7
:1013900010B50A440024C361029B00604060846071
:1013A000C160816141610261036210BD08B582695B
:1013B0004369934201D1826882B9826801328260B6
:1013C0005A1C42611970426903699A4201D3C36889
:1013D0004361002100F0DEFE002008BD4FF0FF3029
:1013E00008BD000070B5202304460E4683F3118823
:1013F000A568A5B1A368A269013BA360531CA361C2
:1014000015782269934224BFE368A361E3690BB1B5
:1014100020469847002383F31188284670BD314643
:10142000204600F0A7FE0028E2DA85F3118870BD9F
:101430002DE9F74F05460F4690469A46D0F81C9086
:10144000202686F311884FF0000B144664B1224623
:1014500039462846FFF73CFF034668B951462846FF
:1014600000F088FE0028F1D0002383F31188A8EB58
:10147000040003B0BDE8F08FB9F1000F03D0019074
:101480002846C847019B8BF31188E41A1F4486F352
:101490001188DBE7C160816141611144C361009B38
:1014A000006040608260016103627047F8B50446E5
:1014B0000E461746202383F31188A568A5B1A368BB
:1014C000013BA36063695A1C62611E7023696269F3
:1014D0009A4224BFE3686361E3690BB120469847F1
:1014E000002080F31188F8BD3946204600F042FE06
:1014F0000028E2DA85F31188F8BD000083694269AB
:101500009A4210B501D182687AB98268013282604C
:101510005A1C82611C7803699A4201D3C3688361B3
:10152000002100F037FE204610BD4FF0FF3010BD07
:101530002DE9F74F05460F4690469A46D0F81C9085
:10154000202686F311884FF0000B144664B1224622
:1015500039462846FFF7EAFE034668B95146284651
:1015600000F008FE0028F1D0002383F31188A8EBD7
:10157000040003B0BDE8F08FB9F1000F03D0019073
:101580002846C847019B8BF31188E41A1F4486F351
:101590001188DBE7026843681143016003B1184713
:1015A000704700001430FFF743BF00004FF0FF33D7
:1015B0001430FFF73DBF00003830FFF7B9BF00001F
:1015C0004FF0FF333830FFF7B3BF00001430FFF7A0
:1015D00009BF00004FF0FF311430FFF703BF0000D8
:1015E0003830FFF763BF00004FF0FF323830FFF7AD
:1015F0005DBF000000207047FFF768BD044B03602B
:10160000002343608360C36001230374704700BFFD
:10161000A040000810B52023044683F31188FFF78B
:101620007FFD02232374002383F3118810BD000083
:1016300038B5C36904460D461BB904210844FFF7B9
:10164000A9FF294604F11400FFF7B0FE002806DACE
:10165000201D4FF48061BDE83840FFF79BBF38BDC7
:10166000026843681143016003B1184770470000E6
:1016700037B5446B41F6A40563591A6811780429FB
:1016800014D1217C022911D11979012312898B40AF
:1016900013420BD101A904F14C0002F075F8645912
:1016A0000246019B2179206800F0ECF903B030BDBF
:1016B000143001F0F9BF00004FF0FF33143001F097
:1016C000F3BF00004C3002F0CBB800004FF0FF3306
:1016D0004C3002F0C5B80000143001F0C7BF000064
:1016E0004FF0FF31143001F0C1BF00004C3002F068
:1016F00097B800004FF0FF324C3002F091B8000074
:1017000070B541F6A4060546825913681978042974
:1017100001D0012070BD017C0229FAD1127901208B
:101720005C8990400440F4D105F1140001F058FFA9
:1017300002460028EDD0AD594FF44073286869790E
:1017400000F08EF9204670BD406BFFF7D9BF000056
:1017500000207047704700007FB5124B012504261A
:10176000044603600023057400F1840243602946A7
:101770008360C3600C4B0290143001934FF44073AC
:10178000009601F009FF094B04F6944229460193A3
:1017900004F14C004FF440730294009601F0D0FF26
:1017A00004B070BDC8400008491700087116000851
:1017B0000A68202383F311880B790B3342F8230046
:1017C0004B79133342F823008B7913B10B3342F872
:1017D000230041F6A403C15002230374002383F3C2
:1017E0001188704738B5037F044613B190F8543020
:1017F000ABB90125201D0221FFF732FF04F11400CF
:1018000025776FF0010100F0D1FC84F8545004F109
:101810004C006FF00101BDE8384000F0C7BC38BD96
:1018200010B5012104460430FFF71AFF0023237787
:1018300084F8543010BD000038B50446002514303B
:1018400001F0C2FE04F14C00257701F091FF201D4C
:1018500084F854500121FFF703FF2046BDE83840CB
:10186000FFF74EBF90F8803003F06003202B19D1B2
:1018700090F88120212A0AD0222A4FF000030ED0AE
:10188000202A0FD1084A42670722826704E0064BEC
:101890004367072383670023C367012070474367BB
:1018A0008367F9E7002070471C22002073B541F6DA
:1018B000A405044643591A681178042919D1017CFA
:1018C000022916D11979012312898B40134210D1B4
:1018D00000F14C06304602F00BF850B101A9304639
:1018E00001F052FF64590246019B2179206800F003
:1018F000C9F802B070BD000001F10B03F7B550F854
:10190000234005460E46F4B1202383F3118805EBEE
:101910008607201D08214C34FFF7A2FEFB685B6997
:101920001B6813B1204601F03DFF01A9204601F0DC
:101930002BFF024648B1019B3146284600F0A2F831
:10194000002383F3118803B0F0BDFB685A69126865
:10195000002AF5D01B8A013B1340F1D105F180022A
:10196000EAE70000133138B550F82140E4B12023F4
:1019700083F3118841F6A403E2581368527903EB0C
:101980008203DB689B695D6845B104216018FFF73D
:1019900067FE294604F1140001F02CFE2046FFF7F3
:1019A000AFFE002383F3118838BD000070470000AC
:1019B00001F00EB9012300F1300200F15001037073
:1019C0000023436042F8043B8A42D361FAD1038189
:1019D0004381704738B50446202383F311880025DE
:1019E00000F10C0300F13002416043F8045B9342C4
:1019F000FBD1204601F00EF90223237085F31188F4
:101A000038BD000070B500EB8103054650690E46F5
:101A10001446DA6018B110220021FFF72DFAA069F0
:101A200018B110220021FFF727FA31462846BDE8F9
:101A3000704001F001BA0000038900F1300200217A
:101A400003F001030381438903F00103438100F1A3
:101A5000100343F8041B9342FBD101F085BA000048
:101A6000F0B4012500EB810447898D40E4683D43D3
:101A7000A469458123600023A2606360F0BC01F08B
:101A8000A1BA0000F0B4012500EB810407898D4064
:101A9000E4683D436469058123600023A2606360BC
:101AA000F0BC01F019BB0000022300F10C0200F1B0
:101AB000300110B5037004460023A0F8883080F888
:101AC0008A3080F88B300381438142F8043B8A429C
:101AD000FBD184F87030204601F042F963681B683E
:101AE00023B120460021BDE81040184710BD00007A
:101AF000037880F88C300523037043681B6810B5A9
:101B000004460BB10421984700232381638110BD53
:101B1000436890F88C201B6802700BB105211847B0
:101B20007047000090F8703070B5044613B1002380
:101B300080F8703004F18002204601F039FA6368C1
:101B40009B6863BB94F8805015F0600615D194F83B
:101B5000813005F07F0545EA032540F202339D42BE
:101B600000F00E815BD8022D00F0DC803FD8002D04
:101B700000F08780012D00F0CF800021204601F089
:101B8000D1FC0021204601F0C1FC63681B6813B141
:101B9000062120469847062384F8703070BD204601
:101BA00098470028CED094F8872094F8863043EAEE
:101BB0000223A26F934238BFA36794F98030A56FC8
:101BC000002B4FF0200380F2FD80002D00F0EC8010
:101BD000092284F8702083F311880021A36F626FBB
:101BE0002046FFF74FFF002383F3118870BDB5F542
:101BF000817F00F0B180B5F5407F49D0B5F5807F99
:101C0000BBD194F88230012BB7D1B4F8883023F0DF
:101C10000203A4F888306667A667E667C3E740F268
:101C200001639D421ED8B5F5C06F3BD2B5F5A06FDC
:101C3000A3D1B4F88030B3F5A06F0ED194F8823000
:101C4000204684F88A3001F0E9F863681B6813B114
:101C50000121204698470323237000236367A3676D
:101C6000E367A0E7B5F5106F32D040F602439D421E
:101C700052D0B5F5006F80D104F18B036367012367
:101C800024E004F18803E56763670223A3678AE71A
:101C900094F88230012B7FF470AFB4F8883043F0B1
:101CA0000203B6E794F885202046616894F88430F2
:101CB0004D6843EA022394F8831094F88220A847E1
:101CC00000283FF45AAF436863670368A367A4E73B
:101CD0002378042B10D1202383F311882046FFF7AB
:101CE000ABFE86F311886368032184F88B601B6860
:101CF00021700BB12046984794F88230002BACD06D
:101D000084F88B300423237063681B68002BA4D0F5
:101D1000022120469847A0E7374B63670223A36759
:101D200000239DE794F88410204611F0800F01F005
:101D30000F010ED001F02EF9012806D002287FF401
:101D40001CAF2E4BA067636767E72D4BA5676367E2
:101D500063E701F011F9EFE794F88230002B7FF48C
:101D60000CAF94F8843013F00F013FF476AF1A06ED
:101D7000204602D501F0EEFB6FE701F0DFFB6CE7D8
:101D800094F88230002B7FF4F8AE94F8843013F08E
:101D90000F013FF462AF1B06204602D501F0C2FBE3
:101DA0005BE701F0B3FB58E7142284F8702083F35B
:101DB00011882B462A4629462046FFF751FE85F317
:101DC000118870BD5DB1152284F8702083F31188ED
:101DD0000021A36F626F2046FFF742FE03E70B224C
:101DE00084F8702083F311882B462A462946204622
:101DF000FFF748FEE3E700BFF8400008F0400008A6
:101E0000F440000838B590F870300446152B29D8F6
:101E1000DFE803F03E28282828283E28280B293907
:101E200028282828282828283E3E90F8871090F84F
:101E30008620836F42EA01229A4214D9C268128A2C
:101E4000B3FBF2F502FB15356DB9202383F311883E
:101E50002B462A462946FFF715FE85F311880A23EB
:101E600084F8703038BD142384F87030202383F355
:101E70001188002320461A461946FFF7F1FD00237A
:101E800083F3118838BDC36F03B198470023E7E798
:101E9000002101F047FB0021204601F037FB636879
:101EA0001B6813B10621204698470623D8E7000097
:101EB00090F87020152A38B5044622D801239340A3
:101EC00040F6416213421DD113F480150FD19B02DD
:101ED00017D50B2380F87030202383F311882B460D
:101EE0002A462946FFF7CEFD85F3118838BDC36821
:101EF0009B695B682BB9C36F03B19847002384F8D3
:101F0000703038BD002101F00DFB0021204601F0AA
:101F1000FDFA63681B6813B1062120469847062323
:101F2000EDE70000024B00221B605B609A60704787
:101F3000AC280020002382680374054B1B68996855
:101F40009142FBD25A68036042601060586070474B
:101F5000AC28002008B5202383F31188037C032BD1
:101F600005D0042B0DD02BB983F3118808BD43692C
:101F700000221A604FF0FF334361FFF7DBFF0023BD
:101F8000F2E790E80C001A6002685360F2E7000084
:101F9000002382680374054B1B6899689142FBD843
:101FA0005A6803604260106058607047AC28002097
:101FB000054B196908741868026853601A60186143
:101FC00001230374FEF700BAAC2800204B1C30B587
:101FD000054687B00A4C10D0236901A8094A00F0D1
:101FE00001F92846FFF7E4FF049B13B101A800F0B4
:101FF0004BF92369586907B030BDFFF7D9FFF8E7FF
:10200000AC280020551F000838B50C4D044641612E
:102010002B6981689A68914203D8BDE83840FFF780
:1020200089BF1846FFF7B4FF01232C6101462374D2
:102030002046BDE83840FEF7C7B900BFAC280020F5
:10204000044B1A681B6990689B68984294BF0020F3
:1020500001207047AC28002010B5084C2368206987
:102060001A6854602260012223611A74FFF790FFFE
:1020700001462069BDE81040FEF7A6B9AC28002053
:10208000FEE7000010B50C4CFFF74CFF00F09CF889
:1020900080220A49204600F021F8012344F8180C58
:1020A000037400F069FC002383F3118862B60448CE
:1020B000BDE8104000F034B8D4280020FC400008EF
:1020C0000441000800F01AB9034B59685A68521AC3
:1020D0009042FBD8704700BF001000E082600222EF
:1020E00002740022427470478368A3F17C0243F8B3
:1020F0000C2C026943F83C2C426943F8382C074AFF
:1021000043F81C2CC268A3F1180043F8102C0222DB
:1021100003F8082C002203F8072C7047E10300089D
:1021200010B5202383F31188FFF7DEFF002104465A
:10213000FFF76AFF002383F31188204610BD0000DB
:10214000024B1B6958610F20FFF732BFAC280020FB
:10215000202383F31188FFF7F3BF000008B5014681
:10216000202383F311880820FFF730FF002383F337
:10217000118808BD49B1064B42681B6918605A6056
:10218000136043600420FFF721BF4FF0FF3070471A
:10219000AC2800200368984206D01A68026050609C
:1021A00018465961FFF7C6BE7047000038B50446AF
:1021B0000D462068844200D138BD036823605C600E
:1021C0004561FFF7B7FEF4E7054B03F114025A61CE
:1021D0009A614FF0FF32DA6100221A62704700BF45
:1021E000AC280020F8B5274F0D4603610446C260B5
:1021F0003E4601F0B5FB3B46022D294653F8142F0D
:1022000038BF02219A421D460AD1386208447C61D7
:10221000BC6122606260A160BDE8F84001F08ABB49
:10222000D7F820E0A0EB0E035F181FD300279068BB
:10223000834217D8376AAA421F44376201D0C01AB6
:10224000906073699A68914219D85A6823606260F5
:1022500014605C60A1609868411A99604FF0FF3388
:10226000F361F8BD97601B1A1268E0E793689F421C
:1022700003D20EEB070001F06DFB3946E1E7891A46
:102280001B68DFE7AC28002038B51B4B01685A6992
:102290001D46904203F114020CD0446821600021D5
:1022A000036893425C60C16025D09A6881680A44E3
:1022B0009A6038BD59614A6000215B69C1609342F0
:1022C00003D1BDE8384001F03FBB9A6881680A44F9
:1022D0009A602C6A01F044FB6A69001B9268824292
:1022E00009D9111A012998BF821C286ABDE8384013
:1022F000104401F02FBB38BDAC2800202DE9F84F69
:10230000204C0027656904F11406B84601F028FB4B
:10231000236AA0EB030AAB6853451DD84FF0200990
:10232000236AAA68D5F80CB013442362AB68AAEB01
:10233000030A2B68B3425E606361EF6001D101F074
:1023400003FB88F311882869D84789F311886569E8
:10235000AB689A45E4D2D9E76369B34210D02062F2
:102360009A68A2EB0A029A60226AAB68821A9B1AE8
:10237000022B2CBFC0180230BDE8F84F01F0EABABA
:10238000BDE8F88FAC28002000207047FEE7000071
:10239000704700004FF0FF3070470000022906D060
:1023A000032906D00129064818BF002070470548B8
:1023B0007047032A9ABF044800EBC2000020704710
:1023C000F0410008A44100082422002070B59AB012
:1023D00006460846144601AD294600F095F8284601
:1023E000FEF742FDC0B2431C5B0086E81800237074
:1023F0000323023404F8013C00231946DAB2023404
:10240000904201D81AB070BDEA5C013304F8011C97
:1024100004F8022CF2E7000008B5202383F31188AA
:102420000348FFF743FA002383F3118808BD00BF78
:10243000682A002010B50446052916D8DFE801F007
:1024400016150316161D202383F311880E4A012149
:10245000FFF7D8FA20460D4A0221FFF7D3FA0C48BD
:10246000FFF7EAF9002383F3118810BD202383F3DB
:1024700011880748FFF7B6F9F4E7202383F31188A2
:102480000348FFF7CDF9EDE7244100084841000873
:10249000682A002038B50C4D0C4C2A460C4904F132
:1024A0000800FFF793FF05F1CA0204F11000094983
:1024B000FFF78CFF05F5CA7204F118000649BDE864
:1024C0003840FFF783BF00BF404300202422002094
:1024D000744100087E4100088941000870B5044637
:1024E00008460D46FEF7C0FCC6B22046013403780C
:1024F0000BB9184670BD32462946FEF79FFC0028EE
:10250000F3D1012070BD00002DE9F84F05460C46BF
:10251000FEF7AAFC2C49C6B22846FFF7DFFF08B138
:102520000536F6B229492846FFF7D8FF08B110361C
:10253000F6B2632E0DD8DFF89080DFF89090244F2C
:10254000DFF894A0DFF894B02E7846B92670BDE885
:10255000F88F29462046BDE8F84F01F077BD252EBB
:102560002ED1072241462846FEF768FC70B9DBF8F9
:10257000003007350C3444F80C3CDBF8043044F8E8
:10258000083CDBF8083044F8043CDDE70822494603
:102590002846FEF753FC98B9A21C0E4B13F8011FF6
:1025A000023209095345C95D02F8041C197801F08B
:1025B0000F01C95D02F8031CF0D118340835C3E7D8
:1025C000267001350134BFE7104200088941000838
:1025D00025420008FFE7F11F0BE8F11F1842000831
:1025E000BFF34F8F044B1A695107FCD1D3F8102168
:1025F0005207F8D1704700BF0020005208B50D4BBC
:102600001B78ABB9FFF7ECFF0B4BDA68D10704D5A9
:102610000A4A5A6002F188325A60D3F80C21D20774
:1026200006D5064AC3F8042102F18832C3F8042112
:1026300008BD00BF9E4500200020005223016745D1
:1026400008B5114B1B78F3B9104B1A69510703D524
:10265000DA6842F04002DA60D3F81021520705D55B
:10266000D3F80C2142F04002C3F80C21FFF7B8FF69
:10267000064BDA6842F00102DA60D3F80C2142F02E
:102680000102C3F80C2108BD9E4500200020005225
:102690000F289ABF00F580604004002070470000BA
:1026A0004FF4003070470000102070470F2808B525
:1026B0000BD8FFF7EDFF00F500330268013204D1BB
:1026C00004308342F9D1012008BD002008BD00007C
:1026D0000F2810B504463FD8FFF782FFFFF78EFFA3
:1026E0001E484FF0FF33072C4361C0F814311DD84A
:1026F0000361FFF775FF230243F02403C360C3683F
:1027000043F08003C36003695A07FCD4FFF768FFF6
:102710002046FFF7BDFF4FF4003100F0F9F8FFF756
:102720008FFF2046BDE81040FFF7C0BFC0F8103152
:10273000FFF756FFA4F108031B0243F02403C0F87F
:102740000C31D0F80C3143F08003C0F80C31D0F8D4
:1027500010315B07FBD4D9E7002010BD00200052E8
:102760002DE9F84F40EA0203054689469046DB060C
:102770005AD122F0030203460244934205D1FFF7E7
:102780003DFF4E46DFF8B8B042E0196801314BD149
:102790000433F2E7264A05F1784326489342264B54
:1027A000264F88BF9A46A3F1FC039CBFDA46184621
:1027B00003F1F80388BF1F46FFF712FF4FF0FF3306
:1027C00006F11C02A5EB060E03603B6843F0020312
:1027D0003B60331FDAF8004014F00504FAD153F8D7
:1027E000041F9A424EF80310F4D1BFF34F8FFFF746
:1027F000F7FE4FF0FF3320223146036028463B6846
:1028000023F002033B6001F011FC58B9203520365B
:10281000A8EB06034B441F2BBCD80120FFF710FF89
:10282000BDE8F88F2046F9E70020BDE8F88F00BF2B
:10283000FFFF0F0014210052102100520C20005203
:102840001020005210B5084C237828B153B9FFF777
:10285000D5FE0123237010BD23B12070BDE81040C8
:10286000FFF7EEBE10BD00BF9E45002002440439B4
:10287000064BD2B210B5904200D110BD441C00B23C
:1028800053F8200041F8040FE0B2F4E7504000583C
:102890000F4B30B51C6F240405D41C6F1C671C6FD4
:1028A00044F400441C670B4C024404392368D2B240
:1028B00043F480732360084B904200D130BD441C28
:1028C00051F8045F00B243F82050E0B2F4E700BFD3
:1028D00000440258004802585040005807B50122F1
:1028E00001A90020FFF7C2FF019803B05DF804FBC7
:1028F00013B50446FFF7F2FFA04206D002A9012259
:10290000002041F8044DFFF7C3FF02B010BD0000E6
:102910000144BFF34F8F064B884204D3BFF34F8F60
:10292000BFF36F8F7047C3F85C022030F4E700BF3D
:1029300000ED00E0034B1B685B0142BF0122024B2C
:102940001A707047D04402589F450020014B1878F8
:10295000704700BF9F450020EFF3098305496833A6
:102960004A6822F001024A6083F30988002383F356
:102970001188704730EF00E0202080F3118862B6A4
:102980000D4B0E4AD96821F4E0610904090C0A4391
:102990000B49DA60CA6842F08072CA60094A0A4983
:1029A000C2F8B01F116841F0010111601022DA77FE
:1029B00083F82200704700BF00ED00E00003FA0535
:1029C000F0ED00E0001000E055CEACC510B52023BE
:1029D00083F311880E4B5B6813F4006314D0F1EE9F
:1029E000103AEFF309844FF08073683CE361094BC0
:1029F000DB68236684F30988FFF722FB10B1064BDE
:102A0000A36110BD054BFBE783F3118810BD00BF28
:102A100000ED00E030EF00E0F3030008F6030008EB
:102A2000F0B5BFF34F8FBFF36F8F1D4B0021C3F87D
:102A30005012BFF34F8FBFF36F8F5A6942F40032C9
:102A40005A61BFF34F8FBFF36F8FC3F88410BFF38A
:102A50004F8FD3F8802043F6E076C2F3C904C2F367
:102A60004E32A507520102EA060E284621464EEADA
:102A70000007013900F14040C3F860724F1CF6D1E5
:102A8000203A12F1200FEED1BFF34F8F5A6942F472
:102A900080325A61BFF34F8FBFF36F8FF0BD00BF1D
:102AA00000ED00E0FEE70000084A094B09498B42AF
:102AB00004D3094A0021934205D3704752F8040F0A
:102AC00043F8040BF3E743F8041BF4E7E84300087A
:102AD000F0460020F0460020F0460020D0F8943068
:102AE000002170B5D0F890404FF0FF359E684A0144
:102AF000A318D3F80009002805DAD3F8000940F03C
:102B00008040C3F80009D3F8000B002805DAD3F899
:102B1000000B40F08040C3F8000B0131A3188E4237
:102B2000C3F80859C3F8085BE1D24FF00113C4F8A9
:102B30001C3870BD00EB81032DE9F04FD3F80CE099
:102B40004F1C4FEA4118DEF814403F03D4F800C090
:102B50006568D0F8902065450AD30120D2F8343852
:102B600000FA01F123EA0101C2F83418BDE8F08F40
:102B7000ACEB0503BEF81060B34228BF334602EB4E
:102B80000806D6F81869B6B2B3EB860F13D8A66854
:102B90003A449946A6F1040A5AF804BFB9F1040F61
:102BA000C2F800B002D9A9F10409F5E71E442B448C
:102BB000A6606360CCE70020BDE8F08F890141F09A
:102BC0002001016103699B06FCD41220FFF77CBA47
:102BD00010B50A4C2046FEF7EDFE094BC4F89030C4
:102BE000084BC4F89430084C2046FEF7E3FE074B30
:102BF000C4F89030064BC4F8943010BDA0450020B6
:102C0000000008405C4200083C46002000000440F0
:102C1000684200080378012B70B505465DD1494B29
:102C2000D0F89040984259D1474B0E216520D3F8F7
:102C3000D82042F00062C3F8D820D3F8002142F037
:102C40000062C3F80021D3F80021D3F8802042F0BD
:102C50000062C3F88020D3F8802022F00062C3F81D
:102C60008020D3F8803000F081FC384BE360384B93
:102C7000C4F800380023D5F89060C4F8003EC023A3
:102C800023604FF40413A3633369002BFCDA0123A0
:102C90000C203361FFF718FA3369DB07FCD41220EC
:102CA000FFF712FA3369002BFCDA00262846A660EB
:102CB000FFF714FF6B68C4F81068DB68C4F8146889
:102CC000C4F81C68002B3AD1224BA3614FF0FF33AC
:102CD0006361A36843F00103A36070BD1E4B98427B
:102CE000C8D1194B0E214D20D3F8D82042F00072E4
:102CF000C3F8D820D3F8002142F00072C3F80021B5
:102D0000D3F80021D3F8802042F00072C3F880206D
:102D1000D3F8802022F00072C3F88020D3F88020FE
:102D2000D3F8D82022F08062C3F8D820D3F800214D
:102D300022F08062C3F80021D3F8003193E7074BFB
:102D4000C3E700BFA04500200044025840140040E3
:102D500003002002003C30C03C460020083C30C04C
:102D6000F8B5D0F89040054600214FF000662046A7
:102D7000FFF724FFD5F8941000234FF001128F685D
:102D80004FF0FF30C4F83438C4F81C2804EB431269
:102D900001339F42C2F80069C2F8006BC2F808090B
:102DA000C2F8080BF2D20B68D5F89020C5F898301D
:102DB000636210231361166916F01006FBD112200E
:102DC000FFF782F9D4F8003823F4FE63C4F8003822
:102DD000A36943F4402343F01003A3610923C4F81B
:102DE0001038C4F814380B4BEB604FF0C043C4F8F4
:102DF000103B094BC4F8003BC4F81069C4F8003913
:102E0000D5F8983003F1100243F48013C5F89820E8
:102E1000A362F8BD3842000840800010D0F890202E
:102E200090F88A10D2F8003823F4FE6343EA0113C5
:102E3000C2F80038704700002DE9F0410EB20D468F
:102E400000EB8608D8F80C100F6807F00303022B7C
:102E500053D0032B53D03F4A3F4F012B18BF174687
:102E6000D0F890404FEA451E002205F1100C04EB0B
:102E70000E03C3F8102B8A69002A42D04A8A05F152
:102E800058033A435B01E2500123D4F81C2803FAAB
:102E90000CF31343C4F81C38A64400234A69CEF847
:102EA000103905F13F03002A3BD00A8A04EB830363
:102EB000898B9208012988BF4A43D0F89810561888
:102EC00041EA02422946C0F8986020465A60FFF75E
:102ED00075FED8F80C301B8A43EA85531F4305F171
:102EE00048035B01E7500123D4F81C2803FA05F5D9
:102EF0001543C4F81C58BDE8F081184FB0E7184FCF
:102F0000AEE704EB4613D3F8002B22F40042C3F8DB
:102F1000002B0123D4F81C2803FA0CF322EA030344
:102F2000B8E704EB83030F4A04EB461629465A60C0
:102F30002046FFF743FED6F80039012223F4004370
:102F400002FA05F5C6F80039D4F81C3823EA05055D
:102F5000CFE700BF00800010008004100080081040
:102F600000800C1000040002D0F894201268C0F811
:102F70009820FFF7B3BD00005831D0F890304901D8
:102F80005B5813F4004004D013F4001F14BF012059
:102F9000022070474831D0F8903049015B5813F453
:102FA000004004D013F4001F14BF0120022070471A
:102FB00000EB8101CB68196A0B6813604B685360A2
:102FC0007047000000EB810330B5DD68AA69136823
:102FD000D36019B9402B84BF402313606B8A1468F7
:102FE000D0F890201C4402EB4110013C09B2B4FB24
:102FF000F3F46343033323F0030343EAC44343F08E
:10300000C043C0F8103B2B6803F00303012B0ED123
:10301000D2F8083802EB411013F4807FD0F8003B5F
:1030200014BF43F0805343F00053C0F8003B02EB61
:103030004112D2F8003B43F00443C2F8003B30BDDC
:103040002DE9F041D0F8906005460C4606EB41139F
:10305000D3F8087B3A07C3F8087B08D5D6F81438AC
:103060001B0704D500EB8103DB685B689847FA0710
:103070002FD5D6F81438DB072BD505EB8403D96898
:10308000CCB98B69488A5E68B6FBF0F200FB12622D
:103090008AB91868DA6890420DD2121A83E81400CF
:1030A000202383F3118821462846FFF78BFF84F302
:1030B0001188BDE8F081012303FA04F26B8923EA49
:1030C00002036B81CB6823B121462846BDE8F0415D
:1030D0001847BDE8F081000000EB81034A0170B59C
:1030E000DD68D0F890306C692668E66056BB1A44FB
:1030F0004FF40020C2F810092A6802F00302012AE6
:103100000AB20ED1D3F8080803EB421410F4807F02
:10311000D4F8000914BF40F0805040F00050C4F8CB
:10312000000903EB4212D2F8000940F00440C2F853
:1031300000090122D3F8340802FA01F10143C3F86F
:10314000341870BD19B9402E84BF4020206020681B
:103150001A442E8A841940F00050013CB4FBF6F466
:1031600040EAC440C6E700002DE9F041D0F8906085
:1031700004460D4606EB4113D3F80879C3F80879E5
:10318000FB071CD5D6F81038DA0718D500EB8103F9
:10319000D3F80CE0DEF81430D3F800C0DA689445B8
:1031A0001BD2A2EB0C024FF000081A60C3F8048097
:1031B000202383F31188FFF78FFF88F311883B06E4
:1031C00018D50123D6F83428AB40134212D0294633
:1031D0002046BDE8F041FFF7ADBC012303FA01F240
:1031E000038923EA02030381DEF80830002BE6D0CE
:1031F0009847E4E7BDE8F0812DE9F047D0F890501A
:1032000004466E69AB691E40F1046E6103D5BDE8EA
:10321000F047FEF749BC002E12DAD5F8003E9A07B7
:1032200005D0D5F8003E23F00303C5F8003ED5F8DD
:103230000438204623F00103C5F80438FEF768FC83
:10324000330505D52046FFF749FC2046FEF750FC24
:10325000B7040CD5D5F8083813F0060FEB6823F443
:1032600070530CBF43F4105343F4A053EB6030078A
:1032700004D56368DB680BB120469847F10200F182
:10328000A180B2020BD5D4F8908000274FF001093D
:10329000D4F89430F9B29B688B4280F0D280F30668
:1032A0001AD5D4F890100A6AC2F30A1702F00F0375
:1032B00002F4F012B2F5802F00F0EB80B2F5402F4F
:1032C0000AD104EB830301F58051DB68186A0023FF
:1032D0001A469F4240F0D1803003D5F8185835D5B2
:1032E000E90303D500212046FFF7AAFEAA0303D570
:1032F00001212046FFF7A4FE6B0303D502212046DF
:10330000FFF79EFE2F0303D503212046FFF798FE0B
:10331000E80203D504212046FFF792FEA90203D557
:1033200005212046FFF78CFE6A0203D506212046C0
:10333000FFF786FE2B0203D507212046FFF780FE0C
:10334000EF0103D508212046FFF77AFE700340F114
:10335000C780E90703D500212046FFF705FFAA072C
:1033600003D501212046FFF7FFFE6B0703D502219D
:103370002046FFF7F9FE2F0703D503212046FFF76C
:10338000F3FEEE0603D504212046FFF7EDFEA80666
:1033900003D505212046FFF7E7FE690603D5062180
:1033A0002046FFF7E1FE2A0603D507212046FFF756
:1033B000DBFEEB0540F1948020460821BDE8F04794
:1033C000FFF7D2BED4F890904FF000084FF0010AFA
:1033D000D4F894305FFA88F79B68BB42FFF451AF92
:1033E00009EB4713D3F8002902F44022B2F5802FED
:1033F00024D1D3F80029002A20DAD3F8002942F09A
:103400009042C3F80029D3F80029002AFBDB394693
:10341000D4F89000FFF7D2FB22890AFA07F322EAD8
:103420000303238104EB8703DB689B6813B13946F0
:103430002046984739462046FFF77CFB08F10108F3
:10344000C6E708EB4112D2F8003B03F44023B3F582
:10345000802F10D1D2F8003B002B0CDA628909FAD8
:1034600001F322EA0303638104EB8103DB68DB6879
:103470000BB12046984701370AE713F0030F00D13C
:103480000A68072B03F101039EBF0270120A013084
:103490001FE704EB830301F58051DA689069026845
:1034A000D0F808C04068A2EB000E002210469742F8
:1034B00008D1DB689B699A683A449A605A68174455
:1034C0005F6009E712F0030F00D10868964502F12A
:1034D000010282BF8CF80000000A0CF1010CE6E743
:1034E000BDE8F08708B50348FFF786FEBDE8084051
:1034F000FFF76CBAA045002008B50348FFF77CFE33
:10350000BDE80840FFF762BA3C460020D0F8903092
:1035100003EB4111D1F8003B43F40013C1F8003B29
:1035200070470000D0F8903003EB4111D1F800391A
:1035300043F40013C1F8003970470000D0F8903010
:1035400003EB4111D1F8003B23F40013C1F8003B19
:1035500070470000D0F8903003EB4111D1F80039EA
:1035600023F40013C1F800397047000000F16043F4
:1035700000F01F020901400903F56143C9B2800050
:1035800083F80013012300F16040934000F561408F
:10359000C0F880310360704730B50433039C01727A
:1035A000002104FB0325C361049B00600363059BAA
:1035B0004060C16042610261856104624262816271
:1035C000C162436330BD00000022416AC2604161B4
:1035D00001616FF001018262C262FEF7E7BD000087
:1035E00003694269934203D1C2680AB1002070475F
:1035F000181D7047036919600021C2680132C2605A
:10360000C269134482699342036124BF436A036120
:10361000FEF7C0BD38B504460D46E3683BB16269AC
:103620000020131D1268A3621344E36238BD237A9D
:1036300033B929462046FEF79DFD0028EDDA38BD56
:103640006FF00100FBE70000C368C269013BC36083
:103650004369134482699342436124BF436A4361CF
:1036600000238362036B03B11847704770B52023B2
:10367000044683F31188866A3EB9FFF7CBFF0546FF
:1036800018B186F31188284670BDA36AE26A13F860
:10369000015B9342A36202D32046FFF7D5FF0023CC
:1036A00083F31188EFE700002DE9F84F04460E463A
:1036B00090469946202787F311880025AA46D4F81A
:1036C00028B0BBF1000F09D149462046FFF7A2FF01
:1036D00020B18BF311882846BDE8F88FA16AA8EBCA
:1036E000050BE36A5B1A9B4528BF9B46BBF1400F65
:1036F0001BD9334601F1400251F8040B914243F8C3
:10370000040BF9D1A36A403640354033A362A26A64
:10371000E36A9A4202D32046FFF796FF8AF31188A4
:103720004545D8D287F31188C9E730465A46FDF798
:103730007BFBA36A5E445D445B44A362E7E7000051
:1037400010B5029C04330172C36103FB0421002302
:1037500000608362C362039B40600363049BC46098
:1037600042610261816104624262436310BD0000F4
:10377000026A6FF00101C260426A42610261002286
:103780008262C262FEF712BD436902699A4203D1A6
:10379000C2680AB100207047184650F8043B0B601D
:1037A00070470000C3680021C2690133C3604369E8
:1037B000134482699342436124BF436A4361FEF725
:1037C000E9BC000038B504460D46E3683BB1236907
:1037D00000201A1DA262E2691344E36238BD237A15
:1037E00033B929462046FEF7C5FC0028EDDA38BD7E
:1037F0006FF00100FBE7000003691960C268013A3D
:10380000C260C269134482699342036124BF436A60
:10381000036100238362036B03B118477047000004
:1038200070B5202304460E4683F31188856A35B9A6
:103830001146FFF7C7FF10B185F3118870BDA36A69
:103840001E70A36AE26A01339342A36204D3E16962
:1038500020460439FFF7D0FF002080F3118870BDA7
:103860002DE9F84F04460D4691469A464FF0200840
:1038700088F311880026B346A76A4FB951462046FF
:10388000FFF7A0FF20B187F311883046BDE8F88F1D
:10389000A06AA9EB0603E76A3F1A9F4228BF1F46AA
:1038A000402F1BD905F1400355F8042B9D4240F8E9
:1038B000042BF9D1A36A40364033A362A26AE36ABB
:1038C0009A4204D3E16920460439FFF795FF8BF350
:1038D00011884E45D9D288F31188CDE729463A465A
:1038E000FDF7A2FAA36A3D443E443B44A362E5E7E8
:1038F000026943699A4203D1C3681BB918467047ED
:103900000023FBE7836A002BF8D0043B9B1AF5D019
:103910001360C368013BC360C3691A4483699A4258
:10392000026124BF436A0361002383620123E5E748
:1039300000F0BAB8034B002258631A610222DA6021
:10394000704700BF000C00400022014BDA60704756
:10395000000C0040014B5863704700BF000C004052
:10396000014B586A704700BF000C00404B68436031
:103970008B688360CB68C3600B6943614B690362EA
:103980008B6943620B6803607047000008B5304BD9
:1039900040F2FF712F48D3F888200A43C3F88820EB
:1039A000D3F8882022F4FF6222F00702C3F88820AF
:1039B000D3F88820D3F8E0200A43C3F8E020D3F8F6
:1039C00008210A43C3F80821234AD3F808311146D5
:1039D000FFF7CCFF214802F11C01FFF7C7FF204889
:1039E00002F13801FFF7C2FF1E4802F15401FFF750
:1039F000BDFF1D4802F17001FFF7B8FF1B4802F13F
:103A00008C01FFF7B3FF1A4802F1A801FFF7AEFFE0
:103A1000184802F1C401FFF7A9FF174802F1E001BD
:103A2000FFF7A4FF154802F1FC01FFF79FFF1448C0
:103A300002F58C71FFF79AFF00F0EAF8114B0522AE
:103A40009A604FF06052DA600F4A1A6108BD00BFF9
:103A50000044025800000258744200080004025852
:103A600000080258000C02580010025800140258B6
:103A700000180258001C0258002002580024025866
:103A80000028025890ED00E01F00080308B500F080
:103A9000BBFAFEF7F7FAFEF74DFFBDE80840FEF768
:103AA000F9BC000070470000114BD3F8E82042F049
:103AB0000802C3F8E820D3F8102142F00802C3F846
:103AC00010210C4AD3F81031D36B43F00803D363B1
:103AD000C722094B9A624FF0FF32DA6200229A61E4
:103AE0005A63DA605A6001225A611A60704700BF57
:103AF000004402580010005C000C0040094A08B560
:103B00001369D1680B40D9B29B076FEA01011161BB
:103B100007D5202383F31188FEF7D4FA002383F31B
:103B2000118808BD000C0040384B4FF0FF31D3F82E
:103B30008020C3F88010D3F880200022C3F88020B2
:103B4000D3F88000D3F88400C3F88410D3F884003D
:103B5000C3F88420D3F88400D86F40F0FF4040F4CD
:103B6000FF0040F43F5040F03F00D867D86F20F08E
:103B7000FF4020F4FF0020F43F5020F03F00D867C2
:103B8000D86FD3F888006FEA40506FEA5050C3F8FE
:103B90008800D3F88800C0F30A00C3F88800D3F87F
:103BA0008800D3F89000C3F89010D3F89000C3F8C1
:103BB0009020D3F89000D3F89400C3F89410D3F871
:103BC0009400C3F89420D3F89400D3F89800C3F875
:103BD0009810D3F89800C3F89820D3F89800D3F839
:103BE0008C00C3F88C10D3F88C00C3F88C20D3F869
:103BF0008C00D3F89C00C3F89C10D3F89C10C3F839
:103C00009C20D3F89C3000F0D3B900BF0044025888
:103C10000122614B1A60614BD3F8F42042F002029A
:103C2000C3F8F420D3F81C2142F00202C3F81C218F
:103C30000222D3F81C315A4BDA605A689104FCD541
:103C4000584A1A6001229A60574ADA6000221A61C3
:103C50004FF440429A61524B9A699204FCD51A681B
:103C600042F480721A604D4B1A6F12F4407F04D0F8
:103C70004FF480321A6700221A671A6842F0010274
:103C80001A60464A134611684807FCD500211161A5
:103C90001A6912F03802FBD1012119604FF08041FE
:103CA00059605A67414ADA62414A1A611A6842F415
:103CB00080321A60394A134611688903FCD51168AD
:103CC00041F4805111601A689204FCD5394A3A498E
:103CD0009A6200225A6319633849DA6399635A6415
:103CE000374A1A64374ADA621A6842F0A8521A60F0
:103CF0002A4B1A6802F02852B2F1285FF9D1482203
:103D00009A614FF48862DA6140221A622E4ADA64BC
:103D10004FF000521A652D4A5A652D4A9A65322293
:103D20002C4B1A601A6802F00F02022AFAD11B4BC0
:103D30001A6942F003021A611A6902F03802182A5D
:103D4000FAD1D3F8DC2042F00052C3F8DC20D3F8DB
:103D5000042142F00052C3F80421D3F80421D3F81F
:103D6000DC2042F08042C3F8DC20D3F8042142F08A
:103D70008042C3F80421D3F80421D3F8DC2042F0B8
:103D80000042C3F8DC20D3F8042142F00042C3F81B
:103D90000421D3F8043170470881005100440258CF
:103DA0000048025800C000F0020000010000FF01BE
:103DB0000088900832306000630207011802030394
:103DC00047040508FD0BFF01000001200010E00082
:103DD00000010100002000524FF0B04208B5D2F8B7
:103DE000883003F00103C2F8883023B1044A136815
:103DF0000BB150689847BDE80840FEF7E7BD00BF2B
:103E0000C02300204FF0B04208B5D2F8883003F04C
:103E10000203C2F8883023B1044A93680BB1D0681A
:103E20009847BDE80840FEF7D1BD00BFC023002081
:103E30004FF0B04208B5D2F8883003F00403C2F85E
:103E4000883023B1044A13690BB150699847BDE823
:103E50000840FEF7BBBD00BFC02300204FF0B042BA
:103E600008B5D2F8883003F00803C2F8883023B1CF
:103E7000044A93690BB1D0699847BDE80840FEF742
:103E8000A5BD00BFC02300204FF0B04208B5D2F856
:103E9000883003F01003C2F8883023B1044A136A53
:103EA0000BB1506A9847BDE80840FEF78FBD00BFD0
:103EB000C02300204FF0B04310B5D3F8884004F47D
:103EC0007872C3F88820A30604D5124A936A0BB10E
:103ED000D06A9847600604D50E4A136B0BB1506B3D
:103EE0009847210604D50B4A936B0BB1D06B9847CA
:103EF000E20504D5074A136C0BB1506C9847A30533
:103F000004D5044A936C0BB1D06C9847BDE81040BF
:103F1000FEF75CBDC02300204FF0B04310B5D3F8CE
:103F2000884004F47C42C3F88820620504D5164A10
:103F3000136D0BB1506D9847230504D5124A936D4C
:103F40000BB1D06D9847E00404D50F4A136E0BB146
:103F5000506E9847A10404D50B4A936E0BB1D06EF6
:103F60009847620404D5084A136F0BB1506F984705
:103F7000230404D5044A936F0BB1D06F9847BDE872
:103F80001040FEF723BD00BFC023002008B5034842
:103F9000FDF718F9BDE80840FEF718BD40240020E1
:103FA00008B5FFF7ABFDBDE80840FEF70FBD000008
:103FB000062108B50846FFF7D9FA06210720FFF7C2
:103FC000D5FA06210820FFF7D1FA06210920FFF7CC
:103FD000CDFA06210A20FFF7C9FA06211720FFF7BC
:103FE000C5FA06212820FFF7C1FA09217A20FFF738
:103FF000BDFA07213220FFF7B9FA0C215220BDE8A3
:104000000840FFF7B3BA000008B5FFF78DFDFDF7D4
:1040100041F8FDF7F1FAFDF7CBFCFDF79BFBFFF74D
:1040200041FDBDE80840FFF783BC000010B5013931
:104030000244904201D1002010BD10F8013B11F85C
:10404000014FA342F5D0181B10BD0000034611F824
:10405000012B03F8012B002AF9D17047121012131B
:1040600012110000682A00204024002053544D33D0
:104070003248373F3F3F0053544D33324837343393
:104080002F373533000000000096000000000000CC
:104090000000000000000000000000000000000020
:1040A00000000000C1150008AD150008E915000862
:1040B000D5150008E1150008CD150008B915000850
:1040C000A5150008F515000800000000CD16000831
:1040D000B9160008F5160008E1160008ED160008EC
:1040E000D9160008C5160008B116000851170008B7
:1040F0000000000001000000000000006D61696E1A
:10410000000000001C410008F0280020682A002060
:1041100001000000812000080000000069646C6557
:10412000000000000200000000000000F918000874
:104130006519000840004000104300202043002083
:10414000020000000000000003000000000000006A
:10415000AD190008000000001000000030430020EE
:10416000000000000100000000000000A045002049
:10417000010102004172647550696C6F7400254240
:104180004F415244252D424C002553455249414C44
:1041900025000000352400089D230008651800084C
:1041A0001924000843000000AC4100080902430044
:1041B000020100C0320904000001020201000524CE
:1041C0000010010524010001042402020524060058
:1041D00001070582030800FF09040100020A00002C
:1041E00000070501024000000705810240000000B1
:1041F00012000000F8410008120110010200004006
:1042000009124157000201020301000004030904DE
:1042100025424F41524425006C756D696E6F757370
:1042200062656535003031323334353637383941DF
:10423000424344454600000000000000251B0008E2
:10424000051E0008B11E000840004000D8460020AE
:10425000D846002001000000E84600208000000051
:104260004001000008000000000100000004000000
:10427000080000000000802A00000000AAAAAAAAE4
:1042800000000000FFFF00000000000000A00A0086
:104290000001400000000000AAAAAAAA0001000034
:1042A000FFFF0000000000000000000010000040C0
:1042B00000000000AAAAAAAA10000040FFFF000008
:1042C00000000000000000000040000000000000AE
:1042D000AAAAAAAA00400000FFFF000000000000F8
:1042E000000000000080024000000000AAAAAAAA64
:1042F00000400140FFFF00000000007007000000C8
:104300000000000000000000AAAAAAAA0000000005
:10431000FFFF00000000000000000000000000009F
:1043200000000000AAAAAAAA00000000FFFF0000E7
:10433000000000000000000000000000000000007D
:10434000AAAAAAAA00000000FFFF000000000000C7
:10435000000000000000000000000000AAAAAAAAB5
:1043600000000000FFFF000000000000000000004F
:104370000000000000000000AAAAAAAA0000000095
:10438000FFFF00000000000000000000000000002F
:1043900000000000AAAAAAAA00000000FFFF000077
:1043A0000000000000000000FF000000000000000E
:1043B0006C4000083F0000005004000077400008F7
:1043C0003F0000000096000000000800040000000C
:1043D0000C42000800000000000000000000000087
:0C43E000000000000000000000000000D1
:00000001FF
